:020000040800F2
:100000000004022001020008990E0008990E000861
:10001000990E0008990E0008990E0008990E000824
:10002000990E0008990E0008990E00085530000836
:10003000990E0008990E0008990E0008990E000804
:10004000990E0008990E0008990E0008990E0008F4
:10005000990E0008990E0008990E0008990E0008E4
:10006000990E0008990E0008990E0008990E0008D4
:10007000990E0008990E0008990E0008990E0008C4
:10008000990E0008990E0008990E0008990E0008B4
:10009000990E0008990E0008990E0008990E0008A4
:1000A000990E0008990E0008990E0008990E000894
:1000B000D9260008990E0008990E0008990E00082C
:1000C000990E0008990E0008990E0008990E000874
:1000D000990E0008990E00085D280008990E000886
:1000E000990E0008990E0008990E0008990E000854
:1000F000990E0008990E0008990E0008990E000844
:10010000990E0008990E0008990E0008990E000833
:10011000990E0008990E0008990E0008990E000823
:10012000990E0008990E0008990E0008990E000813
:10013000990E0008990E0008990E0008990E000803
:10014000990E0008990E0008990E00085124000825
:10015000990E0008990E0008990E0008990E0008E3
:10016000990E0008990E0008990E0008990E0008D3
:10017000990E0008990E0008990E0008990E0008C3
:10018000990E0008990E000871280008990E0008C1
:10019000990E0008990E0008990E0008990E0008A3
:1001A000990E0008990E0008990E0008990E000893
:1001B000990E0008990E0008990E0008990E000883
:1001C000990E0008990E0008990E0008990E000873
:1001D000990E0008990E0008990E0008990E000863
:1001E000990E0008990E0008990E0008990E000853
:1001F000990E0008990E0008990E0008990E000843
:1002000072B6374880F3098836484EF60851CEF268
:100210000001086040F20000CCF200004EF634719C
:10022000CEF200010860BFF34F8FBFF36F8F40F233
:100230000000C0F2F0004EF68851CEF200010860D6
:10024000BFF34F8FBFF36F8F4FF00000E1EE100A46
:100250004EF63C71CEF200010860062080F314884F
:10026000BFF36F8F00F0BEFD02F0B6FB4FF05530CC
:100270001D491E4A91423CBF41F8040BFAE71C4954
:10028000174A91423CBF41F8040BFAE719491A4A50
:100290001A4B9A423EBF51F8040B42F8040BF8E7A0
:1002A00000201749174A91423CBF41F8040BFAE776
:1002B00000F0D8FD02F092FB134C144DAC4203DA6F
:1002C00054F8041B8847F9E700F03EF8104C114D34
:1002D000AC4203DA54F8041B8847F9E700F0C0BDCC
:1002E0000008022000000008000002200004022094
:1002F00000040220F03D00080008022050080220FF
:1003000050080220502B02200002000800020008C2
:1003100000020008000200082DE9F04F2DED108AC0
:10032000C1F80CD0D0F80CD0BDEC108ABDE8F08F2D
:10033000002383F311882846A047002000F0B0FF77
:1003400000F04AFF00DFFEE770B51D4C32230025A8
:1003500023706FF07F061F236570A570E57025710F
:100360006571A571E57125726672A372E57200F080
:1003700057FC20B10F2325726672A372E57202F05A
:1003800085FD104B984217D00133984241F28834D2
:1003900012BF002500240125002002F07DFD0DB1D3
:1003A00000F054F800F0BCFC00F086FB204600F0A2
:1003B000D1F800F04BF8F9E700242546ECE700BF40
:1003C00050080220010007B008B500F0F3FAA0F1D0
:1003D00020035842584108BD07B5054B02211B8830
:1003E000ADF8043001A800F051FB03B05DF804FB48
:1003F0006C3A000810B51148C3680BB100F018FE44
:100400000F4C104A0D4800234FF47A7100F0D4FDD0
:10041000236813B12368013B2360636813B16368E9
:10042000013B6360084B1B7833B9636823B9022032
:1004300000F028FC3223636010BD00BF5C0802207E
:10044000740D0220F5030008700802202DE9F04128
:10045000394C236801336CD0384D394B2A689A42A5
:1004600067D9384B9B6803F1006303F500439A4258
:100470005FD2002000F03AFB334B0220187000F0EE
:10048000F5FB324B1A6C00221A64596C5A64596994
:1004900041F0800159615A61196941F000511961B7
:1004A0001A6172B62A4B1C6024682D68BFF34F8F07
:1004B000BFF36F8F083BC3F88420BFF34F8FD3F88F
:1004C00080205969C2F3C90621F48031C2F34E324B
:1004D00059615201B70743F6E07E02EA0E0838463A
:1004E0003146013948EA000CB1F1FF3FC3F874C24C
:1004F00000F14040F5D1203A12F1200FEDD1BFF3C9
:100500004F8FBFF36F8FBFF34F8FBFF36F8F5A695A
:1005100022F400325A610022C3F85022BFF34F8FF9
:10052000BFF36F8F202383F31188A54684F30888D7
:100530002847BDE8F08100BF008000080480000863
:10054000FF7F000850080220700802200038024097
:1005500008ED00E02DE9F04FB34B8246B3489C68AC
:100560000022C2608FB0202282F31188C2680093FB
:100570000AB100F05DFD0023AD4AAC484FF47A713A
:1005800000F01AFD002383F31188DFF8C0B2BAF13E
:10059000000F01D0CBF800A0A64FCBF80430002507
:1005A0003B702E464FF0FF38012000F05FFBBAF1A0
:1005B000000F00F0C181DBF80030002B40F0BC815F
:1005C0000FB0BDE8F08F0220FFF7FEFE002840F0DC
:1005D000AF81994B1B88ADF82430022109A800F0A7
:1005E00055FAE1E74FF47A7000F0E4F9031E019345
:1005F000EFDB0220FFF7E8FE81460028E9D0019BEF
:10060000581E0428E5D8DFE800F00310131619007F
:100610000EA8052340F8143D042100F037FA4D469A
:1006200000F074FBFFF7D8FE7FE104217E48F4E779
:1006300004218248F1E704218148EEE71C25284681
:1006400000F056FA04350990042109A800F01EFABA
:100650002C2DF4D1E3E7002EBBD0002DB9D0022021
:10066000FFF7B2FE064610B901252E46B1E701207C
:1006700000F03CFA0220387000F0F8FA00255FFA2A
:1006800085F9484600F04AFA0135044618B1484653
:1006900000F054FAF3E7012302203B7000F0D8FA8F
:1006A000009B9B689C4207D2204600F021FA013053
:1006B00040F040810434F3E700243C70CBF8044060
:1006C0003546ADE7002E84D0002D82D00220387050
:1006D00000F0CCFA322000F06DF9051EC4DB15F0F5
:1006E0000306C1D1009A926863199342BCD8B5F54C
:1006F000807FB9D8DFF84C91AE420CDA4FF47A70B3
:1007000000F058F90390039B002BADDB039B06F828
:1007100009300136F0E7C820FFF756FE06460028EC
:10072000A2D02CB9474B4FF0FF32D3F800801A60AB
:10073000444B25F003052544A3EB0409AC42BFD08C
:1007400059F80410204600F0D9F9204600F0D0F9FD
:1007500059F80430984240F0ED800434EEE702206E
:10076000FFF732FE00283FF434AF4FF0000AD146C5
:10077000009B9B689A4537D2BAF1000F17D1B8F1A8
:10078000FF3F14D0CDF824802F494B68A3B100223D
:1007900009A8135C83EA0903DBB2013251F8233064
:1007A000042A83EA1929F4D10AF1040AE0E7504641
:1007B00000F09EF90990E7E71A46082012F0010FB1
:1007C0004FEA52021FBF82F06D4282F4380282F477
:1007D000034282F020020138F0D141F82320013396
:1007E000B3F5807FE8D1D2E70EA8042140F8289D18
:1007F00000F04CF914E70EA8002340F8143D6421E2
:1008000000F010F900287FF4E4AE0220FFF7DCFDD1
:1008100000283FF4DEAE099800F0A2F90EAB43F8D1
:10082000240D04211846E3E7500802205C0802204A
:10083000F5030008700802206E3A000854080220F0
:10084000580802207408022074090220740D022046
:100850000EA8002340F8143D642100F0E3F80028BE
:100860007FF4B7AE0220FFF7AFFD00283FF4B1AE32
:10087000099800F083F90EAB43F8200DD1E7022070
:10088000FFF7A2FD00283FF4A4AE00F07DF90EAB07
:1008900043F81C0DC5E70220FFF796FD00283FF442
:1008A00098AE09A9142000F075F981460EA804211C
:1008B00040F8189D00F0EAF8494609A898E74FF477
:1008C0007A70FFF781FD00283FF483AEB8F1FF3F57
:1008D00005D1FFF781FD354800F0E8FC70E64146A0
:1008E000002000F00BF9002000F002F98045F0D064
:1008F0002F4B6FE60EA8002340F8143D642100F052
:1009000091F800287FF465AE0220FFF75DFD002816
:100910003FF45FAEFFF760FD41F2883000F0C6FCA7
:10092000099800F03FFA00F0F1F94FF0000A3BE6B9
:10093000064675E63546DBE7002000F03BF80390FD
:10094000039B002BFFF633AE012000F081F9039BDF
:10095000213B122B3FF628AE01A252F823F000BF34
:10096000C7050008E505000857060008A9050008A6
:10097000A9050008A9050008C5060008A905000882
:100980005F070008F7070008510800087F08000803
:10099000A905000897080008A9050008BF08000875
:1009A00021060008A9050008F5080008A086010036
:1009B000703A00082DE9F34702AE00244FF47A752F
:1009C00006F8014D144FDFF85880454397F9003081
:1009D0005A1C5FFA84F901D0A34212D158F82400BE
:1009E00003680122D3F81CA031462B46D0470128CA
:1009F00007D10A4B9DF8070083F8009002B0BDE8CC
:100A0000F0870134032CE1D14FF4FA7000F04EFC72
:100A10004FF0FF30F2E700BF00080220980D0220DF
:100A20007C3A00082DE9F0474FF47A75144FDFF84F
:100A3000588006464D43002497F900305A1C5FFA4F
:100A400084F901D0A34210D158F82400036804228D
:100A5000D3F81CA031462B46D047042805D1094BBA
:100A600083F800900020BDE8F0870134032CE3D127
:100A70004FF4FA7000F01AFC4FF0FF30BDE8F08739
:100A800000080220980D02207C3A000830B4074B81
:100A90001A78074B53F8224023689D69054B0A4694
:100AA000AC460146204630BC604700BF980D02208E
:100AB0007C3A0008A086010070B502F00BF9094CE1
:100AC000094E2070002530682378834208D902F04F
:100AD000FBF8336805440133B5F5004F3360F2D3BA
:100AE00070BD00BF990D02207C0D022002F0BAB942
:100AF00000F1006000F500400068704707B502ABE8
:100B000000F1006043F8041D0422194600F500407E
:100B100002F036F903B05DF804FB0000054B1A68DB
:100B2000054B1B781344834202D9104402F0CCB821
:100B3000002070477C0D0220990D022038B5074D2A
:100B400004462868204402F0C7F828B928682044E1
:100B5000BDE8384002F0D8B838BD00BF7C0D022097
:100B600010F0030308D1B0F5806F05D800F10050F4
:100B7000A0F571200068704700207047014BC058F5
:100B8000704700BF20F4F01F014B1868704700BF8A
:100B9000002004E0F0B5204B1E68204B1F885D68E4
:100BA00093F90840C6F30B02BA424FEA164622D028
:100BB0009F89BA4221D01F8BBA4206D102220C244F
:100BC00004FB02335D6893F90840B6F5805F16D0E8
:100BD00041F201039E4208BF5A24421E0A44013DCD
:100BE0000B46934215D215F9016F581C4EB10346BE
:100BF00000F8016CF5E70022E1E70122DFE741247C
:100C0000EBE72C2582421D7001D9981C5C70401ABC
:100C1000F0BD1846FBE700BF002004E004080220F6
:100C2000094B5B88B3F5805F09D041F20102934222
:100C300007D10122054B03EB8203D87870470022CD
:100C4000F8E70020704700BF002004E0743A000875
:100C5000022804D14FF48002034B9A6170470128A7
:100C6000FCD14FF40002F7E700080240022803D14C
:100C70004022034B9A6170470128FCD18022F8E79B
:100C800000080240022805D1064A536983F0400358
:100C9000536170470128FCD1024A536983F08003F5
:100CA000F6E700BF0008024010B50023934203D0CE
:100CB000CC5CC4540133F9E710BD000030B5441ECC
:100CC00014F9010F0B4660B193F90050854201F110
:100CD000010106D11AB993F90020801A30BD013AFA
:100CE000EEE7002AF7D1104630BD00000246034669
:100CF000981A13F9011B0029FAD1704702440346E0
:100D0000934202D003F8011BFAE77047024B1A78AE
:100D1000024B1A70704700BF980D02200008022095
:100D200038B5194C194D204600F0DCFB2946204609
:100D300000F004FC2B681648DA6ED2F8043843F051
:100D40000203C2F8043800F0B1FA1249286800F032
:100D50000FFD2B681048DA6E1049D2F8043823F0E2
:100D60000203C2F80438A0424FF4E1330B6001D013
:100D700000F01EFB0A48A04204D00849BDE83840F4
:100D800000F016BB38BD00BFF8210220D03C00089F
:100D900040420F00183D000830110220800D022053
:100DA0009411022038B50B4B1A780B4B53F82240A4
:100DB0000A4B9C4205460CD0094B002118461822CC
:100DC000FFF79CFF056001462046BDE8384000F073
:100DD000EFBA38BD980D02207C3A0008F8210220B5
:100DE000800D0220F0B5BFF34F8FBFF36F8F1B4B09
:100DF0000021C3F850125A6942F400325A61BFF31D
:100E00004F8FBFF36F8FC3F88410BFF34F8FD3F8AA
:100E10008020C2F3C904C2F34E325201A50743F643
:100E2000E07602EA060E284621464EEA000701391E
:100E3000C3F860724F1C00F14040F6D1203A12F125
:100E4000200FEED1BFF34F8F5A6942F480325A61BE
:100E5000BFF34F8FBFF36F8FF0BD00BF00ED00E019
:100E6000FEE70000084A094B09498B4204D3094AAE
:100E70000021934205D3704752F8040F43F8040B46
:100E8000F3E743F8041BF4E73C3E0008502B022034
:100E9000502B0220502B02201EF0040F0CBFEFF34A
:100EA0000880EFF309808169004A1047B50E0008F9
:100EB00070470000204B02681A60204B42681A609D
:100EC0001F4B82681A601F4BC2681A601E4B026972
:100ED0001A601E4B42691A601D4B82691A601D4BD5
:100EE000C2691A601C4B1D491A681D4B1A601A68AA
:100EF000120A0A701A681B4B1A701B4B1A681B4B9C
:100F00001A601B4B1A681B4B1A601B4B1A681B4B51
:100F10001A601B4B1A681B4B1A601B4B1A681B4B41
:100F20001A601B4B5A6A1B4B1A601B4B1B68DB0772
:100F300001D500BEFEE7FEE7CC0D0220D00D022059
:100F4000D80D0220DC0D0220D40D0220C00D02209D
:100F5000C40D0220C80D022028ED00E0A40D0220DF
:100F6000A80D0220B80D02202CED00E0B00D0220EB
:100F700030ED00E0AC0D02203CED00E09C0D0220C5
:100F800034ED00E0B40D022038ED00E0A00D0220A9
:100F900000ED00E0BC0D0220F0ED00E0054B03F198
:100FA00014025A619A614FF0FF32DA6100221A622C
:100FB000704700BFE00D0220F8B503614FF0804399
:100FC000C2605C6A194B1A46022952F8145F38BF96
:100FD0000221954206461F460AD1586198611C625B
:100FE0000560456081600819BDE8F84000F09CBBD1
:100FF000186AAB68241A0C1902D3E41A2D6804E0AD
:101000009C4202D2204400F09DFBAB689C42F4D885
:101010006B68736035601E606E60B460A9684FF0E5
:10102000FF33091BA960FB61F8BD00BFE00D022082
:1010300010B41B4C234653F8141F814210D0416852
:1010400002680A60026851609A424FF00001C16074
:1010500003D0936881680B4493605DF8044B70473C
:101060000A68626100209A425360C86003D15DF84B
:10107000044B00F061BB93688868034493604FF0B1
:101080008042506A226A821A9342E6D99B1A022B46
:101090002CBFC01802305DF8044B00F053BB00BFFA
:1010A000E00D0220024B00221B605B609A607047DB
:1010B000E00D0220002303748268054B1B689968C9
:1010C0009142FBD25A6803604260106058607047DA
:1010D000E00D022008B5202383F31188037C032B45
:1010E00005D0042B0DD02BB983F3118808BD4369BB
:1010F00000221A604FF0FF334361FFF7DBFF00234C
:10110000F2E790E80C001A6002685360F2E7000012
:10111000002303748268054B1B6899689142FBD8D1
:101120005A6803604260106058607047E00D02200A
:10113000054B19690874186802681A6053601861D1
:1011400001230374FFF7E8B8E00D022030B54B1C13
:1011500087B005460A4C10D023690A4A01A8FFF758
:101160002BFF2846FFF7E4FF049B13B101A8FFF70C
:101170005FFF2369586907B030BDFFF7D9FFF8E773
:10118000E00D0220D510000838B50C4D41612B69E7
:1011900081689A689142044603D8BDE83840FFF759
:1011A00089BF1846FFF786FF01232C61014623748F
:1011B0002046BDE83840FFF7AFB800BFE00D022081
:1011C000044B1A681B6990689B68984294BF002082
:1011D00001207047E00D022010B5084C23682069FB
:1011E0001A6822605460012223611A74FFF790FF8D
:1011F00001462069BDE81040FFF78EB8E00D0220DF
:1012000008B5FFF7DDFF18B1BDE80840FFF7E4BF00
:1012100008BD0000826002220274002242748261D2
:10122000704700008368A3F1840243F8142C02691C
:1012300043F8442C426943F8402C084A43F8242CD4
:10124000C26843F8182C022203F8102C002203F87D
:101250000F2C43F8082CA3F120007047310300083D
:1012600008B5FFF7DFFFBDE80840FFF723BF000028
:1012700010B5202383F31188FFF7D4FF0021044623
:10128000FFF782FF002383F31188204610BD000082
:10129000024B1B6958610F20FFF74ABFE00D022087
:1012A000202383F31188FFF7F3BF000008B5014640
:1012B000202383F311880820FFF748FF002383F3DE
:1012C000118808BD10B5054C2369036058610320DF
:1012D000FFF72EFF2369586910BD00BFE00D022003
:1012E00003682BB10022026059611846FFF7E2BE85
:1012F0007047000049B1064B42681B6918605A608C
:10130000136043600420FFF721BF4FF0FF307047A8
:10131000E00D02200368984206D01A68026050600F
:1013200059611846FFF7C6BE7047000038B504463D
:101330000D462068844200D138BD036823605C609C
:101340004561FFF7B7FEF4E70C3002F01BB900006F
:101350004FF0FF330C3002F015B90000303002F0CE
:10136000B1B900004FF0FF33303002F0ABB90000EC
:101370000C3002F0E1B800004FF0FF310C3002F009
:10138000DBB80000303002F05BB900004FF0FF32F4
:10139000303002F055B9000001F074BA0346034A38
:1013A00043F8042B4360012303727047B43A0008EA
:1013B00010B52023044683F3118801F0B9FA022303
:1013C0002372002383F3118810BD000038B54369F0
:1013D00004460D461BB90421084401F017FE2946B6
:1013E00004F10C0002F08CF8002806DA201D4FF4FE
:1013F0008061BDE8384001F009BE38BD13B5446BCB
:10140000D4F88C341A681178042916D1217A02296B
:1014100013D11979128901238B4013420DD101A9EF
:1014200004F1440001F074FF024630B1D4F88C445A
:10143000019B2179206800F0EBF902B010BD00009B
:101440000C3001F0E3BE00004FF0FF330C3001F030
:10145000DDBE0000443001F0C7BF00004FF0FF3395
:10146000443001F0C1BF00000C3001F0B1BE0000FB
:101470004FF0FF310C3001F0ABBE0000443001F002
:1014800093BF00004FF0FF32443001F08DBF0000E9
:10149000D0F88C2438B5136819780429054601D092
:1014A000012038BD017A0229FAD112795C89012024
:1014B00090400440F4D105F10C0001F043FE0246D7
:1014C0000028EDD0D5F88C544FF4807328686979E2
:1014D00000F08CF9204638BD406BFFF7D9BF000003
:1014E000704700007FB50346114A43F8042B0125DD
:1014F000436002260F4B057204460290019300F1EF
:101500007C02294600964FF480730C3001F0F6FD02
:10151000094B0193029400964FF4807304F52172F5
:10152000294604F1440001F0CFFE04B070BD00BFB5
:10153000D43A0008D9140008FD1300080B682022D3
:1015400082F311880A7903EB820210624A790D3224
:1015500043F822008A7912B103EB82031862022356
:101560000372C0F88C14002383F3118870470000C5
:1015700038B5044601250221043001F047FD04F18D
:101580000C0025756FF00101FFF7D0FE84F84C5078
:1015900004F144006FF00101BDE83840FFF7C6BE1A
:1015A00010B501210446043001F030FD00232375FD
:1015B00084F84C3010BD000038B5044600250C30CE
:1015C00001F0B4FD04F14400257501F095FE201DE5
:1015D00084F84C50012101F019FD2046BDE8384047
:1015E000FFF756BF90F85C3003F06003202B19D151
:1015F00090F85D20212A0AD0222A4FF000030ED055
:10160000202A0FD1084A02650722426504E0064BF2
:101610000365072343650023836501207047036545
:101620004365F9E70020704728080220D0F88C3481
:1016300037B51A681178042904461AD1017A0229AB
:1016400017D11979128901238B40134211D100F16E
:101650004405284601F026FF58B101A9284601F0AB
:1016600057FED4F88C44019B21790246206800F093
:10167000CFF803B030BD000000EB8103F7B51C6A62
:1016800005460E46F4B1202383F3118805EB860747
:10169000201D082101F0BAFCFB685B691B6844341B
:1016A00013B1204601F042FE01A9204601F030FEB0
:1016B000024648B1019B3146284600F0A9F80023B4
:1016C00083F3118803B0F0BDFB685A691268002AE1
:1016D000F5D01B8A013B1340F1D105F15C02EAE72A
:1016E0000D3110B550F82140CCB1202383F311887F
:1016F0000421601801F08AFCD4F88C241368527914
:1017000003EB820304F10C00DB689B69596801F06C
:1017100023FD2046FFF7BCFE002383F3118810BD94
:101720007047000000F0ECBF4FF080430022586388
:101730001A610222DA6070474FF080430022DA60BB
:10174000704700004FF080435863704700F0A4BB1F
:10175000012303700023436000F1240200F13801EB
:1017600042F8043B8A421361FAD1038143817047F6
:1017700038B50446202383F3118800254160C560F5
:10178000056145618561C561056200F099FB022331
:10179000237085F3118838BD70B500EB81030546D1
:1017A0005069DA600E46144618B110220021FFF786
:1017B000A5FAA06918B110220021FFF79FFA31465F
:1017C0002846BDE8704000F055BC0000028902F0D8
:1017D00001020281428902F001024281002202617B
:1017E00042618261C261026200F0D8BCF0B400EBD9
:1017F00081044789E4680125A4698D403D43458102
:1018000023600023A2606360F0BC00F0F3BC000022
:10181000F0B400EB81040789E468012564698D4018
:101820003D43058123600023A2606360F0BC00F0AB
:1018300071BD000070B50223002504460370A0F8B6
:10184000645080F8665080F8675005814581C56016
:10185000056145618561C561056280F84C5000F005
:10186000A7FB63681B6823B129462046BDE870408A
:10187000184770BD436802781B6880F8682005220D
:1018800002700BB10421184770470000436890F8BC
:1018900068201B6802700BB10521184770470000D3
:1018A00070B50023044680F84C3000F15C0200F073
:1018B00097FC63689B685BBB94F85C5015F060060E
:1018C00014D194F85D3005F07F0545EA0325B5F5A0
:1018D000407F00F0A58059D8022D00F0F1803FD85C
:1018E000002D00F08780012D00F0E48000212046CB
:1018F00000F0D4FE0021204600F0C6FE63681B689D
:1019000013B1062120469847062384F84C3070BD59
:10191000204698470028CFD094F8632094F862308E
:1019200043EA0223626D934238BF636594F95C30E9
:10193000656D002B4FF0200380F20181002D00F037
:10194000F080012284F84C2083F311880021636D1C
:10195000226D2046FFF75CFF002383F3118870BDE2
:10196000B5F5807F4DD0B5F5817FBFD194F85E305D
:10197000002BBBD194F8603013F00F0126D01A066B
:10198000204640F1B78000F09DFE1FE0B5F5C06F26
:1019900050D020D840F202339D4200F0AE80B5F521
:1019A000A06FA3D1B4F85C30B3F5A06F0ED194F85A
:1019B0005E3084F86630204600F050FB63681B6898
:1019C00013B1012120469847032323700023236588
:1019D0006365A365A0E7B5F5106F41D040F60243FB
:1019E0009D4267D0B5F5006F80D104F16703236590
:1019F000012333E004F16403236502236365A565D5
:101A00008AE794F85E30012B7FF470AFB4F864304D
:101A100023F00203A4F8643026656665A6657BE7BB
:101A200094F85E30012B7FF461AFB4F8643043F07A
:101A30000203EFE794F86120616894F860304D6824
:101A400094F85F1043EA0223204694F85E20A847EA
:101A500000283FF44BAF4368236503686365DDE707
:101A600094F8672094F85E309A42AFD02378042B24
:101A700010D1202383F311882046FFF7A7FE86F3B9
:101A80001188636884F867601B68032121700BB1BB
:101A90002046984794F85E30002B97D084F8673042
:101AA0000423237063681B68002B8FD0022120461B
:101AB00098478BE72E4B236502236365002388E755
:101AC00094F8601011F0800F204601F00F010ED045
:101AD00000F078FB012806D002287FF407AF254BE1
:101AE000236560659AE7244B2365656596E700F0FA
:101AF0005BFBEFE700F0DCFD68E794F85E30002B5D
:101B00007FF4F4AE94F8603013F00F013FF45EAF51
:101B10001B06204602D500F0C1FD57E700F0B4FDDA
:101B200054E7032284F84C2083F311882B462A467D
:101B300029462046FFF75AFE85F3118870BD5DB136
:101B4000042284F84C2083F311880021636D226DF8
:101B50002046FFF74BFEFFE6052284F84C2083F376
:101B600011882B462A4629462046FFF751FEE3E717
:101B7000FC3A0008F43A0008F83A000838B590F842
:101B80004C300446062B22D8DFE803F03704223716
:101B90003732370090F8631090F86220436D42EAC4
:101BA00001229A4214D9C268128AB3FBF2F502FBF1
:101BB00015356DB9202383F311882B462A46294613
:101BC000FFF726FE85F31188022384F84C3038BDD8
:101BD000032384F84C30202383F3118800231A4612
:101BE00019462046FFF702FE002383F3118838BD13
:101BF000836D03B198470023E7E7002100F04EFD15
:101C00000021204600F040FD63681B6813B10621E7
:101C1000204698470623D8E790F84C20062A38B586
:101C2000044621D80123934013F0670F1DD113F010
:101C300008050FD1DB0617D5052380F84C3020238B
:101C400083F311882B462A462946FFF7E1FD85F3E9
:101C5000118838BDC3689B695B682BB9836D03B17C
:101C60009847002384F84C3038BD002100F016FD61
:101C70000021204600F008FD63681B6813B10621AF
:101C8000204698470623EDE7036F30B500229D6894
:101C9000C46E11464FF0FF3004EB421301329542FF
:101CA000C3F80019C3F81019C3F80809C3F8001BDA
:101CB000C3F8101BC3F8080BEED24FF00113C4F8A1
:101CC0001C3830BD890141F02001016103699B0688
:101CD000FCD4122001F07CB92DE9F04F202387B00D
:101CE0000446C56E83F3118800F17C0305934FF021
:101CF000000B2378012B04D0A36F4BB96B69DB0673
:101D000006D4AB69059843F01003AB61FFF7DAFA2C
:101D10008BF311884FF0000E4FF02009236F9B6862
:101D20005FFA8EF083421BD2202383F31188E0E711
:101D3000E16E0A6A02F4F013B3F5802F66D0B3F5B2
:101D4000402F0DD1C2F30A1602F00F0204EB8202FB
:101D500001F58051D3681F6A00231A469E4248D17C
:101D6000696911F01001E3D1012303FA00F2A36FB6
:101D70001A4200F08C8089F31188AB6823F00103CC
:101D8000AB60A36F23EA0203A36781F3118804EB1E
:101D90008003D3F80C80D8F814100B680093431C10
:101DA0001B030293430104934868009B98425FD24F
:101DB000B8F81060E76E1B1AB34228BF3346049E82
:101DC000BE19D6F81869B6B2B3EB860F62D8029E78
:101DD000BE1903968E680196A6F1040A9C46039EDE
:101DE0005AF8047F3760BCF1040F3BD9ACF1040C06
:101DF000F5E713F0030F08BF0A68072B98BF3A7086
:101E000003F101039CBF120A0137A7E7C2F30A16C8
:101E100002F00F0204EB820201F58051D3689B6946
:101E20001F68D3F808805B68A7EB030C00231F46EC
:101E30009E4208D1D36899698A684B68324433441A
:101E40008A604B608CE713F0030F08BF0F689C4556
:101E500088BF88F8007003F1010384BF3F0A08F1CE
:101E60000108E5E7019E1E4403448E604B609BE73A
:101E7000012189F31188AB6843F00103AB6021B9FC
:101E8000D5F834381A43C5F834288BF311880EF18D
:101E9000010E43E70021ECE710B5074C2046FFF7A1
:101EA00057FC4FF0A0420023E266044AE367226732
:101EB000C4F8803010BD00BF280E0220243B00086B
:101EC00070B50378012B86B005465DD1304BC46EEA
:101ED000984213D12F4B5A6B42F080025A635A69D1
:101EE00042F080025A6100225A610E21432001F023
:101EF0003BFC294BE360294BC4F800380023AB6757
:101F0000C4F8003EC02323604FF40413A363EE6EB5
:101F1000202001F05DF8012333613369DB07FCD435
:101F2000122001F055F83369002BFCDA0026A66078
:101F30002846FFF7A9FE6B68C4F81068DB68C4F890
:101F40001468C4F81C680BBB154BA3614FF0FF333A
:101F50006361D5F880309BB9124B009305F188037B
:101F6000019305F53C7302930223039368460E4BDD
:101F700004930595FFF774F9C5F88000FFF740F961
:101F8000A36843F00103A36006B070BD074BDCE714
:101F9000280E0220003802404014004003002002B6
:101FA000003C30C0303B0008D91C0008083C30C061
:101FB000F8B5C46E054600212046FFF783FE296F61
:101FC00000234FF001128F68C4F834384FF00066D8
:101FD000C4F81C284FF0FF3004EB431201339F423A
:101FE000C2F80069C2F8006BC2F80809C2F8080B11
:101FF000F2D20B686B676362EB6E10221A611E6986
:1020000016F01006FBD1122000F0E2FFD4F80038E1
:1020100023F4FE63C4F80038A36943F4402343F07B
:102020001003A3610923C4F81038C4F81438094B0D
:10203000EB60094BC4F8106BC4F8003BC4F810699E
:10204000C4F800396B6F03F1100243F480136A6720
:10205000A362F8BD003B000840800010C26E90F8FB
:102060006610D2F8003823F4FE6343EA0113C2F885
:10207000003870472DE9F0410EB200EB86080D469E
:10208000D8F80C100F6807F00303022B50D0032B75
:1020900050D03D4A3D4F012B18BF1746C46E4FEA42
:1020A000451E04EB0E030022C3F8102B8A6905F1CC
:1020B000100C002A40D04A8A05F158035B013A43CC
:1020C000E2500123D4F81C2803FA0CF31343A6446E
:1020D0004A69C4F81C380023CEF8103905F13F03D3
:1020E000002A39D00A8A898B9208012988BF4A437D
:1020F000416F04EB8303561841EA024246672946C2
:102100005A602046FFF7DEFDD8F80C301B8A43EA00
:1021100085531F4305F148035B01E7500123D4F8C1
:102120001C2803FA05F51543C4F81C58BDE8F081D6
:10213000174FB3E7174FB1E704EB4613D3F8002B63
:1021400022F40042C3F8002BD4F81C28012303FA20
:102150000CF322EA0303BAE704EB83030E4A5A6046
:1021600004EB461629462046FFF7ACFDD6F80039A9
:1021700023F40043C6F80039D4F81C38012202FACF
:1021800005F523EA0505CFE7008000100080041064
:102190000080081000800C1000040002026F12681A
:1021A0004267FFF771BD00005831C36E49015B58AB
:1021B00013F4004004D013F4001F14BF01200220C8
:1021C000704700004831C36E49015B5813F400406A
:1021D00004D013F4001F14BF012002207047000038
:1021E00000EB8101CB68196A0B6813604B68536080
:1021F0007047000000EB810330B5DD68AA69136801
:10220000D36019B9402B84BF402313606B8A1468D4
:10221000C26E1C44013CB4FBF3F46343033323F06C
:10222000030302EB411043EAC44343F0C043C0F848
:10223000103B2B6803F00303012B09B20ED1D2F837
:10224000083802EB411013F4807FD0F8003B14BF34
:1022500043F0805343F00053C0F8003B02EB4112BF
:10226000D2F8003B43F00443C2F8003B30BD00000D
:102270002DE9F041264DEE6E06EB40130446D3F8EF
:10228000087BC3F8087B38070AD5D6F81438190735
:1022900006D505EB84032146DB6828465B68984732
:1022A000FA0733D5D6F81438DB072FD514B995F8CB
:1022B0004C305BB305EB8403D968CCB98B69488A91
:1022C0005E68B6FBF0F200FB12628AB91868DA6841
:1022D00090420DD2121A83E81400202383F3118850
:1022E0000B482146FFF786FF84F31188BDE8F08193
:1022F000012303FA04F26B8923EA02036B81CB68A2
:1023000023B121460248BDE8F0411847BDE8F081FD
:10231000280E022000EB810370B5DD68C36E6C6986
:102320002668E6604A0156BB1A444FF40020C2F802
:1023300010092A6802F00302012A0AB20ED1D3F86A
:10234000080803EB421410F4807FD4F8000914BF8E
:1023500040F0805040F00050C4F8000903EB4212F6
:10236000D2F8000940F00440C2F80009D3F834085C
:10237000012202FA01F10143C3F8341870BD19B902
:10238000402E84BF4020206020682E8A841940F0AF
:102390000050013C1A44B4FBF6F440EAC440C6E7DE
:1023A0002DE9F041284CE66E06EB40130546D3F8C4
:1023B0000879C3F80879F9071AD5D6F81038DA077A
:1023C00016D504EB8003D9684B691868DA68904227
:1023D0002CD2121A4FF000081A60C3F80480202390
:1023E00083F3118829462046FFF794FF88F311886C
:1023F0003B0619D5D6F83428012303FA05F5154212
:1024000012D0202383F31188A36F10482B43A367B6
:10241000D6F8343823EA0505C6F834580021FEF70B
:102420005FFF002383F31188BDE8F081012303FAE5
:1024300005F2238923EA020323818B68002BD7D07E
:10244000294620469847D3E7280E0220A40E0220F2
:102450002DE9F74F8A48C46E6669A3691E4016F4D9
:10246000805F6661054608D000238367FFF7E2F9C5
:1024700003B0BDE8F04F00F0FFBD002E12DAD4F833
:10248000003E7F4899071EBFD4F8003E23F00303A7
:10249000C4F8003ED4F8043843F00103C4F804380B
:1024A000FFF7F4F9320504D500237548AB67FFF751
:1024B000E1F9B3040CD5D4F8083813F0060FE3683B
:1024C00023F470530CBF43F4105343F4A053E36060
:1024D000370704D56B68DB680BB169489847F00291
:1024E00062D4B1020CD5D5F86C80DFF894A1002736
:1024F0004FF001092B6F9B68F9B28B4280F0A380EB
:10250000F2060DD5202383F31188A3695D4823F0DB
:102510001003A3610021FEF7E3FE002383F311887B
:102520003303D4F818481DD5E70302D50020FFF780
:102530009FFEA50302D50120FFF79AFE600302D596
:102540000220FFF795FE210302D50320FFF790FE3E
:10255000E20202D50420FFF78BFEA30202D505207C
:10256000FFF786FE770383D5E60702D50020FFF745
:1025700017FFA50702D50120FFF712FF600702D55C
:102580000220FFF70DFF210702D50320FFF708FF08
:10259000E20602D50420FFF703FFA3067FF568AF2C
:1025A0000520FFF7FDFE63E7D5F86CA0DFF8D4B097
:1025B0004FF000092B6F9B685FFA89F7BB4290D3FD
:1025C0000AEB4713D3F8002902F44022B2F5802F1A
:1025D00036D1D3F80029002A32DAD3F8002942F0A4
:1025E0009042C3F80029D3F80029002AFBDB3946C2
:1025F000E86EFFF767FB01232A89BB406FEA0308F7
:1026000008EA02022A8105EB8702D268926822B1A9
:1026100039461B4801939047019B202282F3118881
:10262000DAF8342808EA0202CAF83428AA6F00212E
:1026300013435846AB67FEF753FE002383F311881C
:1026400009F10109B6E708EB4112D2F8003B03F4A7
:102650004023B3F5802F10D1D2F8003B002B0CDAC9
:102660006A8909FA01F322EA03036B8105EB81030E
:10267000DB68DB680BB15046984701373AE700BF8B
:10268000280E0220A40E0220C36E03EB4111D1F8E4
:10269000003B43F40013C1F8003B7047C36E03EBEB
:1026A0004111D1F8003943F40013C1F800397047E3
:1026B000C36E03EB4111D1F8003B23F40013C1F8C2
:1026C000003B7047C36E03EB4111D1F8003923F48E
:1026D0000013C1F8003970474FF0804310B51A69F4
:1026E000920708D500241C61202383F3118800F091
:1026F00035FC84F31188BDE8104000F0BDBC00003B
:102700000E4A136C43F0010313640D4A936843F0BF
:10271000010393604FF080436B229A624FF0FF32C7
:10272000DA6200229A615A63DA605A6001225A61C1
:1027300008211A601C2001F017B800BF00380240C1
:10274000002004E0024A136843F0800313607047DE
:1027500000440040024A136843F08003136070474E
:10276000007800402DE9F041466D3768F569356223
:102770000446280719D015F0080F0CBF002180214E
:10278000EA0748BF41F02001AB0748BF41F04001D4
:10279000680748BF41F48071202383F31188201D0E
:1027A00000F034FC002383F31188EA050AD52023C6
:1027B00083F311884FF40071201D00F027FC0023E3
:1027C00083F31188AB060CD5202383F31188736A39
:1027D00094F85C1020461940FEF7F8FD002383F3BF
:1027E0001188380616D5290614D5202383F31188BD
:1027F00004F1300000F04CFF002825DA0821201DEC
:1028000000F004FC27F0C00343F0400333600023D2
:1028100083F311886A060ED5202383F31188626C36
:10282000A36C9A4201D1A36B83B927F040073760AC
:10283000002383F31188EB060DD5226E136953B183
:102840005069BDE8F0411847B062E0E71021201D53
:1028500000F0DCFBE9E7BDE8F081000008B50348C3
:10286000FFF780FFBDE8084000F006BC30110220F1
:1028700008B50348FFF776FFBDE8084000F0FCBB51
:102880009411022037B51F4C1F4D2046FEF786FDE0
:10289000009404F10C0000234FF480621B4900F007
:1028A00021FE4FF48062009404F13000184B194966
:1028B00000F0BAFE184B6365A565184C0B21262065
:1028C00000F052FF2046FEF769FD04F10C00009471
:1028D00000234FF48062124900F004FE04F130003E
:1028E0000094104B10494FF4806200F09DFE0F4B96
:1028F00063650B215220A56503B0BDE8304000F0B0
:1029000033BF00BF3011022080F93703F8110220D5
:1029100045270008F81902200044004094110220C5
:10292000F815022055270008F81D02200078004005
:10293000204B002908BF1946037A0166012B10B508
:1029400007D11D4B984226D11C4A136C43F4003327
:102950001364426D0C68836DB3FBF4F3D3608B6832
:1029600043F040035360CB6843F0010393604B682E
:1029700043F4967141F0010111604FF0FF31116293
:102980005A0505D513F010230DD0B3F1805F0ED09A
:1029900080F85C1010BD0A4B9842DAD1074A136CDC
:1029A00043F08043D4E77F2380F85C3010BD3F23A1
:1029B000FAE700BF3C3B000830110220003802401B
:1029C0009411022000207047FEE7000070470000CD
:1029D0004FF0FF307047000000F006BF08B500F070
:1029E00079FB00F075FABDE8084000F0F9B8000086
:1029F00070470000022906D0032906D001290648A5
:102A000018BF0020704705487047032A9ABF044842
:102A100000EBC20000207047743D0008283D00080C
:102A20003008022070B5044608460D46FEF75EF9F0
:102A3000C6B22046013403780BB9184670BD324641
:102A40002946FEF73BF90028F3D1012070BD0000B4
:102A50002DE9F04F80469BB008460C461646FEF71F
:102A600045F93A49C5B22046FFF7DCFF08B1023DFF
:102A7000EDB237492046FFF7D5FF08B11035EDB26A
:102A8000632D01AF0CD8DFF8D490DFF8D4A03D4619
:102A900094F800B0BBF1000F1CD185F800B003E042
:102AA0002146384600F084FF3846FEF71FF9C0B2D1
:102AB000431C5B0088E848003370032373700023D5
:102AC00002361946DAB2904206F1020636D81BB039
:102AD000BDE8F08FBBF1250F2BD107221B49204603
:102AE000FEF7ECF840B9DAF800302B609AF80430C1
:102AF0002B7107340535CBE7082215492046FEF730
:102B0000DDF8B0B91349AB1C11F8012F100902F020
:102B10000F0210F8090012F8092003F8012C0E4AE0
:102B200003F8020C914203F10203EDD11835083489
:102B3000AEE785F800B001340135A9E7FA5C06F884
:102B4000022C06F8011C0133BCE700BFD83C00088A
:102B5000E03C00081FF4F01F2BF4F01FEF3C0008CE
:102B6000E93C000808B5202383F311880348FEF7E9
:102B70005DFD002383F3118808BD00BFF82102200A
:102B800010B50446052916D8DFE801F0161503161E
:102B9000161D202383F311880E4A0121FEF7FCFD48
:102BA00020460D4A0221FEF7F7FD0C48FEF704FD12
:102BB000002383F3118810BD202383F31188074875
:102BC000FEF7D6FCF4E7202383F311880348FEF7D1
:102BD000E7FCEDE7883C0008AC3C0008F821022047
:102BE00038B50C4D0C4C0D492A4604F10800FFF78E
:102BF0002FFF05F1CA0204F110000949FFF728FF71
:102C000005F5CA7204F118000649BDE83840FFF71F
:102C10001FBF00BFB826022030080220003D000878
:102C20000A3D0008E03C0008BFF34F8F024AD3681A
:102C3000DB03FCD4704700BF003C024008B5074BE3
:102C40001B7853B9FFF7F0FF054B1A69002ABFBF85
:102C5000044A5A6002F188325A6008BD16290220DF
:102C6000003C02402301674508B5054B1B7833B98A
:102C7000FFF7DAFF034A136943F00043136108BD0D
:102C800016290220003C02400B2870B513D80B4ACD
:102C90000B4C137863B90B4E4FF0006144F82310CE
:102CA00056F8235001330C2B2944F7D1012313701C
:102CB00054F8200070BD002070BD00BF48290220DC
:102CC00018290220943D0008014B53F8200070475A
:102CD000943D00080C2070470B2810B5044601D91C
:102CE000002010BDFFF7D0FF064B53F824301844E6
:102CF000C21A0BB9012010BD12680132F0D1043B99
:102D0000F6E700BF943D00080B2810B504462FD805
:102D1000FFF78AFFFFF792FF1649F323CB60FFF717
:102D200083FFC300DBB243F4007343F002030B6183
:102D30000B6943F480330B61FFF776FFFFF7A4FFC5
:102D40000D4B53F824300344BFF34F8F0B4A984286
:102D50000AD3BFF34F8FBFF36F8FFFF785FF204676
:102D6000BDE81040FFF7B8BFC2F85C022030EEE7C4
:102D7000002010BD003C0240943D000800ED00E042
:102D80002DE9F047D40715464DD41318B3F1026F5F
:102D900049D2324B1B68DA0745D5314CFFF74EFF5D
:102DA000F323E360FFF740FF2F46401A40F201296A
:102DB000032F884601EB000618D8294C40F2011970
:102DC0007B1A4344012B01EB000623692FD823F023
:102DD00001032361FFF748FF2846BDE8F087366806
:102DE00051F8043CB34218D1043FE1E7B307E4D102
:102DF000236923F440732361236943EA09032361B0
:102E00000431D8F800303360BFF34F8FFFF70CFF69
:102E1000E368002BE3D0F323E360236923F001038D
:102E20002361FFF721FF4FF0FF30BDE8F08723F467
:102E300040732361236943EA090323618A4631F819
:102E4000023B3380BFF34F8FFFF7EEFE3688BAF8B0
:102E50000030B6B2B342B3D0DFE700BF0038024063
:102E6000003C0240084908B50B7828B153B9FFF778
:102E7000E5FE01230B7008BD23B1BDE808400870D2
:102E8000FFF7F2BE08BD00BF16290220014B186DE6
:102E9000704700BF00280040094B1A6F120407D486
:102EA0001A6F42F400721A671A6F42F400421A67EE
:102EB000044A136843F480731360034B186570472A
:102EC000003802400070004000280040FEE700008B
:102ED00010B51A4CFEF7E6F8FEF760F800F0AAF815
:102EE000802217492046FEF795F9012344F8180C73
:102EF0000374144B144AD96821F4E0610904090CE5
:102F00000A431249DA60CA6842F08072CA60104A05
:102F10001049C2F8B01F116841F001011160102280
:102F2000DA77202283F82220002383F3118862B607
:102F30000948BDE81040FEF79BB900BF080E02200B
:102F4000C43D000800ED00E00003FA05F0ED00E0EC
:102F5000001000E055CEACC5CC3D00082DE9F8438B
:102F60001A4C4FF0804300256769586A04F1140831
:102F70002E46226ABB68811A8B420CD96169414591
:102F800022D013441B1A022B2CBFC0180230BDE8FC
:102F9000F843FEF7D7BB134423623B68D7F80C9085
:102FA000C3F8048043456361FD6001D1FEF7C4FBB3
:102FB00086F311883869C847202383F311884FF0BE
:102FC00080436769586AD4E7BDE8F883E00D0220C2
:102FD000034B59685A68521A9042FBD8704700BF99
:102FE000001000E083691943037C81610A2B03D13F
:102FF0004369194205D170470B2B06D143698B43B6
:1030000003D100234361FEF755B8704770B50468DB
:1030100005460E46AC4200D170BDE3683343E36021
:1030200016B12269134203D0A1686068FFF7DAFF86
:103030002468EFE7034B044A1A60044B044A1A6001
:10304000704700BF4C2B0220502B0220482B02203F
:103050000000082080B5074A536823F0010300AF41
:103060005360EFF30983683383F30988002383F304
:10307000118880BD30EF00E098B5202300AF83F3C6
:103080001188104B5B6813F4006318D0F1EE103A0E
:10309000EFF309844FF0807344F84C3C0A4BDB6833
:1030A00044F8083CA4F1680383F30988FEF788F824
:1030B00018B1064B44F8503C98BD054BFAE783F332
:1030C000118898BD00ED00E030EF00E041030008FA
:1030D0004403000808B500F05DFB074800F00CFC55
:1030E000FEF75AF9FEF732FBFEF7FAF9FFF780FC1C
:1030F000BDE80840FEF716BB543B000830B5039C02
:103100000172043304FB0325C361049B03630021A4
:10311000059B00604060C16042610261856104629C
:1031200042628162C162436330BD00000022416A95
:1031300041610161C2608262C2626FF00101FEF70B
:10314000F5B8000003694269934203D1C2680AB12D
:1031500000207047181D704703691960C26801326A
:10316000C260C269134482690361934224BF436A07
:1031700003610021FEF7CEB838B504460D46E3687A
:103180003BB16269131D1268A3621344E36200201D
:1031900038BD237A33B929462046FEF7ABF800281C
:1031A000EDDA38BD6FF00100FBE70000C368C269CB
:1031B000013BC3604369134482694361934224BF66
:1031C000436A436100238362036B03B1184770476E
:1031D00070B52023044683F31188866A3EB9FFF751
:1031E000CBFF054618B186F31188284670BDA36A47
:1031F000E26A13F8015BA362934202D32046FFF711
:10320000D5FF002383F31188EFE700002DE9F74F86
:103210001F4604460E469146202383F311884FF043
:1032200080480025D8F82430FB18009307F1FF3AB6
:10323000AB46A36AABB91AF1030F06D9394620464B
:10324000FFF79AFF68B1002305E0D8F82410009A30
:10325000511A8F42F3D283F31188284603B0BDE898
:10326000F08FA16AE36AA9EB05025B1A934228BFBB
:103270001346402B1CD9334601F1400251F8040B90
:1032800043F8040B9142F9D1A36A40334036A3625C
:103290004035A26AE36A9A4202D32046FFF786FFCE
:1032A0008BF311884D45D8D2202383F31188C0E7D2
:1032B0001A4630460193FDF7F7FC019BA26A1A44B7
:1032C0001E44A2621D44E4E710B5029C017204335F
:1032D00003FB0421C36100238362C362039B036376
:1032E000049B00604060C4604261026181610462CD
:1032F0004262436310BD0000026AC260426A4261DA
:10330000026100228262C2626FF00101FEF70EB814
:10331000436902699A4203D1C2680AB1002070472A
:10332000184650F8043B0B6070470000C368C26940
:103330000133C3604369134482694361934224BFEC
:10334000436A43610021FDF7E5BF000038B504463C
:103350000D46E3683BB123691A1DA262E26913447A
:10336000E362002038BD237A33B929462046FDF7B1
:10337000C1FF0028EDDA38BD6FF00100FBE7000067
:1033800003691960C268013AC260C2691344826964
:103390000361934224BF436A036100238362036B8A
:1033A00003B118477047000070B5202304460E464D
:1033B00083F31188856A35B91146FFF7C7FF10B14D
:1033C00085F3118870BDA36A1E70A36AE26A013397
:1033D0009342A36204D3E16920460439FFF7D0FF8A
:1033E000002080F3118870BD2DE9F74F1F46044679
:1033F0000D469146202383F311884FF08048002624
:10340000D8F82430FB18009307F1FF3AB346A36ABB
:10341000ABB91AF1030F06D939462046FFF796FFDC
:1034200068B1002305E0D8F82410009A511A8F42A1
:10343000F3D283F31188304603B0BDE8F08FA06A61
:10344000E36AA9EB06021B1A934228BF1346402BDE
:103450001CD905F1400355F8042B40F8042B9D427C
:10346000F9D1A36A4033A3624036A26AE36A9A4262
:1034700004D3E16920460439FFF782FF8BF31188FA
:103480004E45D8D2202383F31188C0E71A46294637
:103490000193FDF709FC019BA26A1A441D44A26234
:1034A0001E44E2E7026943699A4203D1C3681BB92B
:1034B000184670470023FBE7836A002BF8D0043BD3
:1034C0009B1AF5D01360C368013BC360C3691A44FB
:1034D000836902619A4224BF436A036100238362C5
:1034E0000123E5E710B50A440024C361029B006094
:1034F00040608460C160816141610261036210BD0E
:1035000008B582694369934201D1826882B98268B1
:10351000013282605A1C42611970426903699A4201
:1035200001D3C36843610021FDF7F4FE002008BD0C
:103530004FF0FF3008BD000070B5202304460E4652
:1035400083F31188A568A5B1A368A269013BA360B4
:10355000531CA36115782269934224BFE368A361D9
:10356000E3690BB120469847002383F3118828466E
:1035700070BD31462046FDF7BDFE0028E2DA85F336
:10358000118870BD2DE9F04F1E4685B004460F46E8
:103590009046D0F81C90202383F311884FF080428E
:1035A0000025526A0293B2180192AA4606F1FF3B27
:1035B000A3680BB3A368013BA360A369591CA16175
:1035C0001B783B702369A169994224BFE368A3611A
:1035D0007A1CB9F1000F03D003922046C847039A22
:1035E0008AF31188B8F1010805F1010518D0029B92
:1035F00083F311881746DBE71BF1030F07D9314628
:103600002046FDF777FE0028D2D0002306E04FF0D9
:103610008042516A019A511A8E42F1D283F3118885
:10362000284605B0BDE8F08FC16081614161C3618A
:103630001144009B0060406082600161036270473A
:10364000F8B504460E461746202383F31188A56873
:10365000A5B1A368013BA36063695A1C62611E7037
:10366000236962699A4224BFE3686361E3690BB12D
:1036700020469847002080F31188F8BD394620463F
:10368000FDF738FE0028E2DA85F31188F8BD000066
:10369000836942699A4210B501D182687AB9826819
:1036A000013282605A1C82611C7803699A4201D3FC
:1036B000C36883610021FDF72DFE204610BD4FF049
:1036C000FF3010BD2DE9F04F1E4685B004460F4671
:1036D0009046D0F81C90202383F311884FF080424D
:1036E0000025526A0293B2180192AA4606F1FF3BE6
:1036F000A3680BB3A368013BA36063695A1C6261B2
:103700003978197023696169994224BFE36863615C
:103710007A1CB9F1000F03D003922046C847039AE0
:103720008AF31188B8F1010805F1010518D0029B50
:1037300083F311881746DBE71BF1030F07D93146E6
:103740002046FDF7D7FD0028D2D0002306E04FF039
:103750008042516A019A511A8E42F1D283F3118844
:10376000284605B0BDE8F08F00F1604300F01F026D
:10377000400903F5614309018000C9B200F16040CE
:1037800083F8001300F5614001239340C0F88031B5
:1037900003607047124B00211A694FF0FF321A6123
:1037A000196158695A615961186A60F0805018624D
:1037B0001962586A5A620B4A5962106840F4807064
:1037C0001060186F00F44070B0F5007F1EBF4FF41A
:1037D000803018671967536823F40073536070478B
:1037E0000038024000700040354B364A1A64364AB1
:1037F0004FF4404111601A6842F001021A601A68E1
:103800009207FCD59A6822F003029A609A689A603F
:103810002B4B19469A6812F00C02FBD1186800F085
:10382000F90018609A601A6842F480321A600B68D6
:103830009B03FCD54B6F43F001034B67204B5A6F42
:103840009007FCD5214A5A601A6842F080721A60CB
:103850001D4B1A4659684904FCD5196841F480315A
:1038600019605368D803FCD5136843F40033136020
:10387000154A53689903FCD5114B1A689201FCD57F
:10388000134A9A6040F20112C3F88C200022C3F858
:103890009020104A40F2093111609A6842F0020209
:1038A0009A60074B9A6802F00C02082AFAD15A6C07
:1038B00042F480425A645A6E42F480425A6670471B
:1038C0000038024000040010007000400836400933
:1038D00000948838003C02404B6843608B688360EA
:1038E000CB68C3600B6943614B6903628B694362B8
:1038F0000B68036070470000214B0246186B10B53F
:1039000040F2FF7420431863196D1E482143196566
:103910001146FFF7E1FF1C4802F11C01FFF7DCFF35
:103920001A4802F13801FFF7D7FF194802F1540194
:10393000FFF7D2FF174802F17001FFF7CDFF1648DD
:1039400002F18C01FFF7C8FF144802F1A801FFF74C
:10395000C3FF134802F1C401FFF7BEFF114802F193
:10396000E001FFF7B9FF104802F1FC01FFF7B4FFD7
:103970000E4802F58C71BDE81040FFF7ADBF00BFE7
:1039800000380240000002400004024000080240EB
:10399000000C0240001002400014024000180240D7
:1039A000001C024000200240002402400028024087
:1039B00080EA0102844612F0030F4FD111F0030F89
:1039C00032D14DF8044D11F0040F51F8043B0BD0E7
:1039D000A3F101329A4312F0803F04BF4CF8043B3C
:1039E00051F8043B16D100BF51F8044BA3F101324A
:1039F0009A4312F0803FA4F101320BD14CF8043B02
:103A0000A24312F0803F04BF51F8043B4CF8044B32
:103A1000EAD023460CF8013B13F0FF0F4FEA3323A3
:103A2000F8D15DF8044B704711F0010F06D011F882
:103A3000012B0CF8012B002A08BF704711F0020F70
:103A4000BFD031F8022B12F0FF0F16BF2CF8022B5B
:103A50008CF8002012F47F4FB3D1704711F8012B7E
:103A60000CF8012B002AF9D1704700BF1210121375
:103A7000121100000010410001105A00F82102202C
:103A8000301102209411022053544D3332463F3FEF
:103A90003F3F3F3F0053544D333246375B347C3514
:103AA0005D780053544D333246375B367C375D7852
:103AB0000000000065130008511300088D13000872
:103AC0007913000885130008711300085D130008BE
:103AD000491300085D140008491400088514000803
:103AE000711400087D1400086914000855140008BA
:103AF0004114000800000000010000000000000068
:103B000000000000A11800087D1B0008191C000817
:103B1000400040001811022018110220010000008E
:103B20002811022080000000400100000500000074
:103B30007573625F70756D70000000000096000084
:103B40000000000000000000000000000000000075
:103B5000000000000000802A00000000AAAAAAAA13
:103B600000000000FFFF00000000000000A00A00AD
:103B70000000000000000000AAAAAAAA000000009D
:103B8000FFFF0000000000000000000000500000E7
:103B900000000000AAAAAAAA00000000FFFF00007F
:103BA000000000000000000080290000000000006C
:103BB000AAAAAAAA80140000FFFF000000707007E4
:103BC000000000000000020000000000AAAAAAAA4B
:103BD00000000100FFFF00000000000008000000DE
:103BE0000020000000000000AAAAAAAA00100000FD
:103BF000FFFF0000000000080000000000000000BF
:103C000000000000AAAAAAAA00000000FFFF00000E
:103C100000000000000000000000000000000000A4
:103C2000AAAAAAAA00000000FFFF000000000000EE
:103C3000000000000000000000000000AAAAAAAADC
:103C400000000000FFFF0000000000000000000076
:103C50000000000000000000000000000000000064
:103C60000000000000000000000000000000000054
:103C70000000000000000000000000000000000044
:103C80000000000000000000020000000000000032
:103C900079160008E116000840004000882602203E
:103CA000982602200200000000000000030000002F
:103CB00000000000211700080000000010000000B4
:103CC000A826022000000000010000000000000003
:103CD000280E02200101020025424F4152442500D6
:103CE0002553455249414C2500666D7576350030A7
:103CF0003132333435363738394142434445460052
:103D00004172647550696C6F740025424F41524492
:103D1000252D424C00000000812B0008F5290008E9
:103D2000E5150008652B000843000000303D000841
:103D300009024300020100C032090400000102022E
:103D400001000524001001052401000104240202E1
:103D50000524060001070582030800FF090401008D
:103D6000020A000000070501024000000705810269
:103D700040000000120000007C3D0008120110010C
:103D800002000040830440570002010203010000CA
:103D9000040309040080000000800000008000008F
:103DA0000080000000000200000004000000040089
:103DB00000000400000004000000040000000400F3
:103DC000000004006D61696E00000000E43D000821
:103DD00050290220482B022001000000CD2E0008AF
:103DE0000000000069646C65000000000000000035
:103DF000FF00000000000000883A00083F000000BB
:103E000049040000953A00083F00000051040000FA
:103E1000A33A00083F0000000096000000000800E0
:103E200004000000903D00080000000000000000B9
:103E30000000000000000000000000000000000082
:00000001FF
